:1000000003308A008E2B0000FF00030E8301A10045
:100010000A08A0008A010408A2007708A300780853
:10002000A4007908A5007A08A600831383120B1E8A
:100030001B288B182C28220884002308F70024088A
:10004000F8002508F9002608FA0020088A00210E89
:100050008300FF0E7F0E09008A110A1237280A104A
:100060008A100A11820728340C3401340634013016
:10007000A8068B108A110A121B28D437ED30731092
:10008000D0307636E931E5350000432B552A201073
:100090002019B018B2173218B1190000CE30F03262
:1000A000F434BA1235173333202B00005039EF3AAD
:1000B000641DA51AAE1966104900CE30F032F43432
:1000C000BA1235173333202B0001CE30E2376A1DC8
:1000D000A51AAE19661049003F308400831300084A
:1000E00003197F280230F800F701F70B7528F80B89
:1000F00074289730F700F70B7B28800B72280800D4
:1001000045188428061385280617831606138312BC
:10011000C5188C2886128D2886168316861283129F
:10012000451994280612952806168316061283127E
:10013000C5199C2808129D280816831608128312D8
:10014000861783168613A4288312861383168613B4
:1001500083120800C308031DAF288713B028871730
:10016000A7132708831687008312C40E4408C5000E
:100170008020C40E4408C50080201A30F700F70B19
:10018000BF28000008001430BF006C208713A7139D
:10019000270883168700831286138316861383121B
:1001A000B1013108023C031CDD280230BF006C2085
:1001B0000330C5008020B10AD1281A30F700F70BB0
:1001C000DF2800000230C50080201A30F700F70B4E
:1001D000E7280000B1013108023C031CFB2831086C
:1001E0002F20B200C3013208C400AA200230BF0091
:1001F0006C20B10AEB28080001303F02C100400822
:10020000023C031D05294030C10741088038C20067
:10021000C3014208C400AA2008003E080C3A031992
:100220001B29063A03192329073A03192929053AF4
:1002300003192E293329C3010130C400AA2002303A
:10024000BF006C203F290130BF000230C000FC20FD
:100250003F290130BF00C000FC203F29C3011030FE
:10026000C400AA203F293E081F3C031C392907303F
:10027000BE050130C3003E08C400AA203F29080083
:10028000831603178C170C140000000083120C084F
:100290007F39031984290313B10003170D080313D1
:1002A000B20003170F080313B3003108BE000D217D
:1002B000320803178D000313330803178F008316CA
:1002C0008C170C140000000083120C0D0E0D7F39EA
:1002D000031984290313B10003170D080313B20097
:1002E00003170F080313B3003108BE000D213208B5
:1002F00003178D000313330803178F008D0A0319AA
:100300008F0A031340290317031308008E30F700E8
:100310003208F8003108F900FA01F808031D9A299B
:100320007908F800F9010830F702F808031D9A2946
:10033000F701A2290310F81BA129F90DF80DF70305
:100340009A29F8130800831603178C170C14000061
:1003500000000318D22983120C087F390313B2005E
:1003600003170D080313B30003170F080313B4009A
:100370003208BE000D21330803178D000313340823
:1003800003178F0083168C170C14000000008312D3
:100390000313B10BCC29CF2983160317D229F129D6
:1003A0008316031783120C0D0E0D7F390313B20051
:1003B00003170D080313B30003170F080313B4004A
:1003C0003208BE000D21330803178D0003133408D3
:1003D00003178F008D0A03198F0A03100313B10B43
:1003E000A3290800F701F801F901FA01C601C701C4
:1003F000C801C90145084404430442040319302AD2
:100400002030CA000310BE0DBF0DC00DC10DC60DBA
:10041000C70DC80DC90D45084902031D192A440816
:100420004802031D192A43084702031D192A4208DE
:100430004602031C2A2A4208C6024308031C430F33
:10044000C7024408031C440FC8024508031C450F9B
:10045000C9020314F70DF80DF90DFA0DCA0B022AA3
:1004600046308400831308000408B6003508B8003D
:100470000319C62A3408C1003308C0003208BF007F
:100480003108BE00C501C4012030C3008230C20063
:100490003E080319B82AC60042080319B82AC6073D
:1004A0000318592A7F30C602031CB82A0319B82A38
:1004B0005D2A8130C6070318B82A4608F700F801FC
:1004C000F901FA013F08CA00CA174008C9004108EB
:1004D000C8001830C600C701481C862A4508FA071C
:1004E000031C782AF90A031D782AF80A0319C7178A
:1004F0004408F907031C7F2AF80A0319C7174308A1
:10050000C000C0174008F8070318C717C70DF80C3C
:10051000F90CFA0CCA0CC90CC80C0310C60B6B2AD8
:100520000130F7070318B82AF81B9D2ACA0DFA0DE7
:10053000F90DF80DF7030319B82ACA1FAE2AFA0AF3
:10054000031DAE2AF90A031DAE2AF80A031DAE2ABE
:10055000F80CF90CFA0CF70A0319B82A3F08C7007F
:100560004308C706C71FB62AF817BC2AF813BC2AC7
:10057000F701F801F901FA017A08B4007908B3002B
:100580007808B2007708B100B80B3A2A3408C100E5
:100590003308C0003208BF003108BE003E08B63C38
:1005A000BE00FA013F08C200BF170310BF0CC00C09
:1005B000C10CFA0CF90CF80CF70CBE0BD52AC21FB3
:1005C000EC2AF709F809F909FA09F70A0319F80AF0
:1005D0000319F90A0319FA0A7A08B4007908B30072
:1005E0007808B2007708B100B41F032BB603B61623
:1005F000B109B209B309B409B10A0319B20A03195E
:10060000B30A0319B40A3B30BD009A30BC00CA30AB
:10061000BB00BA010A30B80035080319B60A34081D
:10062000C1003308C0003208BF003108BE003D08D9
:10063000C5003C08C4003B08C3003A08C200F221D0
:100640000008B100840A0008B200840A0008B30060
:10065000840A0008B400FD308407F708031D432B0B
:10066000350A38020319432B36080319452B0F3975
:10067000380203193D2B0318752BB61B752B361B3F
:10068000452B2030712B2030B605B61E532BB612E9
:100690003508031DB6037708B6002D30BE000D21C6
:1006A0003608F700B60135083802031D612B7708BC
:1006B000B6002E30BE000D213608F7002030B605FA
:1006C00000303030B61E712BB6123508031DB6034C
:1006D0007708B6002D30BE000D213608F700B601B0
:1006E0003030F7077708BE000D213D08C1003C08F7
:1006F000C0003B08BF003A08BE00C501C401C301E9
:100700000A30C200F2217A08BD007908BC007808DE
:10071000BB007708BA00B80B0F2B080084018313C5
:100720001F308305713083168F000F088312281045
:10073000831603170908C039890003131F129F127B
:100740000030031788008312870188018901FF3078
:100750000313A7000B16C0308B0483160113031775
:100760000908C039890003131F129F12283003178C
:1007700088000908C039890003131F129F1229300D
:1007800003178800831203131F179F1383169F13E9
:1007900083121F149412A71227088316870083124E
:1007A00027162708831687008312A71127088316A8
:1007B00087000130831294000030831694000108F2
:1007C000C73908388100831290010030F800920088
:1007D000003083169200831227152708831687009E
:1007E0008312970183169B019C0101309D008312A7
:1007F00003178701880189017130831603138F0065
:100800000F088312C3200130BF00C000FC203D3020
:1008100003178D0000308F00031340210130BF000B
:100820000230C000FC20453003178D0000308F00DF
:10083000031340210430B100FA30BF006C20B10B2B
:100840001C2CC3200030F8001F08C33978049F0017
:100850009F140130BF006C209F182C2C9F149F18F0
:100860002F2C1E08B201B10086217A08AC0079084D
:10087000AB007808AA007708A9000430F8001F0828
:10088000C33978049F009F140130BF006C209F186B
:10089000472C9F149F184A2C1E08B201B1008621D4
:1008A0007A08B0007908AF007808AE007708AD008C
:1008B000281C9E2C0130BF00C000FC204E300317C6
:1008C0008D0000308F00031007300313B100A32107
:1008D000043084002C08B4002B08B3002A08B200AE
:1008E0002908B1000330B50034222030BE000D21AC
:1008F0005630BE000D210130BF000230C000FC2088
:10090000563003178D0000308F000310063003139C
:10091000B100A321043084003008B4002F08B300D4
:100920002E08B2002D08B1000330B500342220306B
:10093000BE000D214930BE000D21E12C0130BF0069
:10094000C000FC205D3003178D0000308F000310C5
:1009500007300313B100A321043084002C08B40035
:100960002B08B3002A08B2002908B1000330B500F3
:1009700034222030BE000D215630BE000D21013042
:10098000BF000230C000FC20653003178D0000302E
:100990008F00031006300313B100A321043084003C
:1009A0003008B4002F08B3002E08B2002D08B100A3
:1009B0000330B50034222030BE000D214930BE0086
:1009C0000D210230B100FA30BF006C20B10BE32CD6
:0409D000212C630073
:04400E00F52CFF3F4F
:00000001FF
